:020000040000FA
:02000000CF2807
:020008007D2D4C
:10001000C60000300D28C6004030C70047207C30A5
:10002000502047085020460850204C201820080037
:100030000A30C1001B28C10B1A2808002830672588
:10004000383008203930082014300820703008205B
:10005000563008206C300820C8306725383008201A
:100060000C30082001300820013067255825080091
:1000700043208A110A12C50A0319C40A003E031953
:1000800008000B20382844088A004508820005141F
:1000900085148510051008000514851085140800C6
:1000A000C8000830C9008510C81B85140514051048
:1000B000C80DC90B5328831685148312051400003C
:1000C000051083168510831208008207003401345E
:1000D00003340434063407342A342A3420345334A5
:1000E00074346F3470342D340034573461347434C4
:1000F0006334683420342A342A3400345634653466
:100100007234203431342E343034313400342034DD
:100110006234793420344D342E3459342034003450
:10012000543469346D346534203453346534743454
:100130000034303430343A34303430343A343034BB
:1001400030340034533474346134723474342034B1
:100150004F346E3400344D3465346D3420344F34B4
:1001600076346534723400344D3465346D34203463
:1001700044346934733470340034083444345734AC
:100180004E34203455345034073400342A342A3461
:1001900020342034203420342A342A340034031309
:1001A0008312850107309F00831620308500BE3002
:1001B0008600483081000C1083120F309000C03050
:1001C0008B008511051205118514051423251E20A9
:1001D0000C3008200230BC00803008200030C40001
:1001E0006C30C5003820C0300820382077257725AE
:1001F000803008203820C030082038207725772527
:10020000BC0BEC280130082077257725A001A1013F
:10021000A201AC01B201B301803008200030C4005B
:100220009030C5003820B21B1829C0300820382073
:1002300022250D300820B201AD012D086520C038FF
:100240000820861C3421861D5821061D9421061A7B
:100250001D295E25061A1D290C300820B310861EA4
:10026000B314061E3129512A5E25861855292430DB
:100270002002031C4829861E41292D0803194A29FA
:1002800044292D08031D50290516E6240512552979
:10029000861E5029AD0A06302D020318AD015529DE
:1002A000AD032D0A05300319AD00861C5529080041
:1002B0005E2586199129861E7E292D0C0339203E44
:1002C00084002D18722910308007F0300005BD0021
:1002D0002D083030031D60303D020F3003188005BB
:1002E000000E7A29800A0F300005093CF030031C0B
:1002F000800500080F3930380B209129E2210318BE
:100300008A29DF2405165E250512DF2405165E25E1
:10031000051291290516E62405125E250516ED2421
:100320000512861D912908005E250619DF29861E03
:10033000BC292D0C0339203E84002D18AE29F03045
:1003400000050319A72910308002000EB8292D08D6
:100350002030031D50308007000EB8290F300005F3
:100360000319B52980030008B8290930800700085F
:100370000F3930380B20DF2905302C02031CC5292A
:10038000AC01A901AA01AB01CD292C083C22AC0A81
:1003900029082A042B040319AC012908A0002A0803
:1003A000A1002B08A2007F30B000C030E322DF2480
:1003B00085155E258511DF2485155E258511061DB1
:1003C000DF2908002C08BD002430200203181D2A54
:1003D000200821042204031403191D2AAC012C084F
:1003E0003C2229082A042B040319142A2908200670
:1003F000031D032A2A082106031D032A2B082206AF
:10040000031403191D2AAC0A05302C02031CEF2922
:100410000130AC002C083C222C032022AC0A053011
:100420002C02031C0A2AAC032008A9002108AA00F8
:100430002208AB002C08202203103D08AC00080065
:1004400083169B009B079B0721309B078312293053
:1004500084000330BC00000883169A001C15553038
:100460009D00AA309D009C149C18342A9B0A83127C
:10047000840ABC0B2B2A080083169B009B079B0752
:1004800021309B078312293084000330BC0083167F
:100490001C141A089B0A83128000840ABC0B472A8A
:1004A000080000308E0080308F0083160C148312F9
:1004B000B201B701803008200030C400A230C5006E
:1004C00038203318642A22253310321A882AB21CA5
:1004D000762A2308A9002408AA002508AB002F08C3
:1004E000B21A7F30B0008030E322B210321CA42A4E
:1004F0002008A9002108AA002208AB002E08B21E7D
:10050000832AB2127F30B000C030E3223210A42A16
:10051000B21AA42A0C233503031D952A2308A90027
:100520002408AA002508AB009F2AB503C623B50AF4
:10053000E9232608A9002708AA002808AB007F3075
:10054000B000C030E322B216861E3523B21B0C2940
:10055000B21DAC2A321D432C3C303702031C642AE6
:10056000BD223219B72A32147F30AE005A2A321413
:10057000B2147F30AE00AF00642AE624051662256F
:100580000512ED248510051005150B108B15630061
:100590003318D82A321D2E0832192F08B000B01D8A
:1005A000C72A0516B31CD824B31862250512C72A1A
:1005B0000511851405141E200C3008208515DF2434
:1005C0008511B7010800BD00B00C0630BC00B00CAE
:1005D000031CEC2ABC0BE72A3C0865203D040820DC
:1005E0003C0C0339293E84003C18FB2A000E0F39CD
:1005F00030380B20BC0A00080F3930380B20BC0AF9
:10060000840A06303C020319082B3A300B20F62AE4
:100610000800013008206625803008200030C40022
:10062000C630C50038208330082035081C2339081F
:100630000B203A080B200800BB003B30840022232B
:10064000222308000830BC00BD010310BB0DBD0D06
:10065000F6303D070318BD000318BB0ABC0B252B61
:1006600084033D083038800008005E25861A962BEA
:10067000861C6E2B061A962B32194C2B80300820C4
:100680000030C4009930C5003820A301A401A501A1
:10069000B50132152C25722BB21D502B32117D2B3A
:1006A0008030B4009723031C752BC0300820003025
:1006B000C400AB30C50038200430BC00E624051669
:1006C0005E250512BC0B5E2B1430BC00622505169E
:1006D0005E250512BC0B662BB215722B83160C100F
:1006E0008312B217861E722B942BDF2485155E258C
:1006F0008511DF2485155E25851185303402031CA4
:100700008C2BB215B4014225C6232908A3002A0860
:10071000A4002B08A500B214861E7D2B321D942B3D
:100720003216B2120330B800B401B7010800230832
:10073000A9002408AA002508AB001A3035020318C6
:10074000A52BA03084003508B72B2A3035020318BA
:10075000AF2B8317203084001A303502B72B3A3084
:1007600035020318C52B4A3084002A30350284072D
:100770008407840729088000840A2A088000840AE4
:100780002B0880008313B50A031008001B303502C4
:100790000318CE2BA03084003503DC2B2B30350220
:1007A0000318D82B8317203084001B303502DC2B34
:1007B0004A3084002B303502840784078407000800
:1007C000A900840A0008AA00840A0008AB00831369
:1007D000080025080F39BD002B080F39BD0203188A
:1007E000F42B0A30BD0703103D08A800250E0F3971
:1007F000BD002B0E0F39031C013EBD020318032C54
:100800000630BD0703103D0EA80424080F39BD00B3
:100810002A080F39031C013EBD020318122C0A30AE
:10082000BD0703103D08A700240E0F39BD002A0E96
:100830000F39031C013EBD020318212C0630BD07F1
:1008400003103D0EA70423080F39BD0029080F39F6
:10085000031C013EBD020318322C0A30A31A0430D7
:10086000BD0703103D08A600230E0F39BD00290E59
:100870000F39031C013EBD020318402C0330BD0795
:100880003D0EA6040800803008200030C400B430BB
:10089000C5003820C0300820382022253508B60091
:1008A000B5013213861EA624B21B582A061EC72481
:1008B000321B612C3C3037020318842C331D522C20
:1008C000952C33116225C623350303196D2C290895
:1008D000A3002A08A4002B08A5007F30B0008030B8
:1008E000E322350303197E2CB503C623B50AE92399
:1008F0002608A9002708AA002808AB007F30B0000E
:10090000C030E3223213522CBD2280300820003048
:10091000C400B430C50038203310622506083039D1
:10092000303A031D8E2C3315B315321C522C20087F
:10093000A9002108AA002208AB002E08B3197F30B5
:10094000B000C030E322B3113210522C5E25861A5B
:10095000C62C861CB72C35080319B32CB50A360AE9
:100960003502031CB52C0130B5000923C22C200828
:10097000A9002108AA002208AB007F30B000C030D7
:10098000E322B217861EC22C3217B70108005E257B
:10099000061AD72C35080319D02CB503031DD22C09
:1009A0003608B5000923061ED32C3217B7010800FC
:1009B0000C30BE00C0002630BF006430102D09305E
:1009C000BE00C0001C30BF006430102D2630BE00B9
:1009D000C0000B30BF006430102D2630BE00C000B8
:1009E0000B30BF00FA30102D1330BE00C0000530B0
:1009F000BF00C830102D0F30BE00C0000830BF004F
:100A0000C830102D0C30BE00C0002630BF00C830EA
:100A1000102D0930BE00C0001C30BF00C830102DA2
:100A2000C2003830810042088B1667258B120800FF
:100A3000C3003830810043088B16672543086725BB
:100A40008B1208002325D82485155E258511DF2407
:100A500085155E25851108008515F424851160250E
:100A60000516FB24051260258515022585116025D4
:100A700005160930BE00C0001C30BF00C830182564
:100A80000512080085150925851160250516022522
:100A9000051260258515FB24851160250516133088
:100AA000BE00C0000530BF00C83018250512080080
:100AB0002730C1005B2DC10B5A2D08001E30672D59
:100AC0003230672D6430672DC830672D0130C20089
:100AD000DD30C1006B2D6C2D6D2DC10B6A2D00001A
:100AE000712D722DC20B682D08000530782D0A304B
:100AF000C3006225C30B792D0800FC00030EFD0026
:100B00000A08FE000408FF000B19902D0C189F2DF9
:100B10000B188B2DB92D0B108B11B7013314B92D78
:100B20000B11C00B9C2D3F08C0000000C00B952D81
:100B3000013086063E08C00038308100B92D0C1007
:100B400000308E0080308F002230C2253108AE0088
:100B50003214B70A321DB92DB219B52D2530C22570
:100B60003108AF00B214B41BB40A321AB80BB92D55
:100B700032127F0884007E088A007D0E8300FC0EFE
:100B80007C0E09008400B101B114E325311C08007A
:100B9000311560300002031C0800B1158001840388
:100BA000E325311C0800311660300002031C0800E8
:100BB000B11680018403E325311724300002031CA1
:100BC0000800800108003110800A00080F390A3C33
:0C0BD000031D08003114063080070800E7
:02400E00023F6F
:1042000043006F0070007900720069006700680069
:1042100074002000280043002900200032003000F4
:104220003200300020006200790020004D002E0096
:10423000590061006D0061006D006F0074006F0037
:10424000FF0000000000000000000000000000006F
:10425000000000000000000000000000000000005E
:00000001FF
